:100A5D00232132303045465500232432303045466F
:020A6D00550032
:1009EA00AF8475840F758A83E4F58475C04475CF26
:0509FA00E4C2C38F847C
:0109FF0022D5
:0609B0008F27AD27AF26E2
:0209B6008D1E94
:1009B80012098EEFC454F0F51FAF1E12098EEF25F1
:0409C8001FF51FFFF9
:0109CC002208
:100967008F828E83D3E5829DE5839C501943B7011F
:10097700758F03E4F0F58F53B7FE2582F582740473
:060987003583F58380DEDC
:01098D002247
:0206D800A90770
:1006DA0020C3FD20C5FAC2C4D2C5E4FFFC30C3FD65
:1006EA0030C3FDE5C154F8FA64086003BA1011E595
:1006FA001DBF01044401800254FEF5C27C01807CC6
:10070A00BA180B851CC27C02C2C4C2C5806EBA204C
:10071A00028038EA64287030B9010CBC02028015E4
:10072A00EC6404701F8019BC02088BC27C03C2C52A
:10073A008012BC03088DC27C04C2C58007BC0404B5
:10074A00D2C57F01C2C48034BA300AD2C4D2C57CB1
:10075A0009E4FF8027BA3802801EBA4006C2C2C224
:10076A00C58019BA48028010BA50028003BA5808E4
:10077A00D2C47C08AEC28004D2C4D2C5C2C3EC645F
:08078A000860030206EAAF0655
:010792002244
:100A8000AE05AD078E1C8B1DE4FB7F011206D8223C
:100A6F00AE03AB05AD078E1C751DA07F021206D815
:010A7F002254
:0603B2008B3D8A3E893FED
:1003B8007547FF75480A75495D75440175450075AF
:1003C8004600E4F543F542F541F540E47F50FEFD73
:1003D800FCAB43AA42A941A840C312066C5031AFF6
:1003E800437BA0E4FD120A807844E475F00112060C
:1003F800C8EF12064DAF43AE42AD41AC40E47B01BD
:10040800FAF9F812065F8F438E428D418C4080BB0B
:10041800AB47AA48A949120607FF900000E06F7091
:1004280062900001120620FF900001E06F70549066
:100438000002120620FF900002E06F704690000351
:10044800120620FF900003E06F7038900004120637
:1004580020FF900004E06F702A900005120620FF2C
:10046800900005E0B5071C900006120620FF9000DA
:1004780006E0B5070E900007120620FF900007E07F
:100488006F60037F0022AB3DAA3EA93F120607FF1B
:10049800900011E06F702A900001120620FF900072
:1004A80012E0B5071C900002120620FF900013E02E
:1004B800B5070E900003120620FF900014E06F604D
:1004C800037F0022900009E0F55BA3E0F55DA3E05F
:1004D800F55E900019E0F557A3E0F559A3E0F55A49
:0204E8007F0192
:0104EA0022EF
:0D09CD008F0DAF18AE17120A348E178F1859
:0209DA00AC0669
:0D09DC00AB07AF04AD07AF03AB58120A80A4
:0109E90022EB
:0E0A9000E55CC3955B500605580558055C22D1
:100A34000FBF00010ED3EF955EEE955D4006120ADE
:050A440090E4FEFF221A
:040277008E088F0955
:10027B00E4F50DF50EF513F514F515F516F517F563
:10028B0018855917855A18855758F50EF50D755C55
:10029B0001E4F512E50D643A6016AF18AE171209BA
:1002AB00DA8F0DAF18AE17120A348E178F1880E441
:1002BB000514E51470020513AF18AE171209DA1204
:1002CB0009CD8F0EAD0EAF0D1209B68F1085101222
:1002DB001209CF1209CD8F0EAD0EAF0D1209B675E7
:1002EB0015008F16EF2512F512E516751600F5158C
:1002FB001209CF1209CD8F0EAD0EAF0D1209B6EF4D
:10030B00421685150A85160BE5162512F5121209EC
:10031B00CF1209CD8F0EAD0EAF0D1209B68F0FE5B3
:10032B000F2512F512E50F705CF50CE50CC395105B
:10033B0050531209CF1209CD8F0EAD0EAF0D12090E
:10034B00B68F11E5112512F512C3E50B9509E50AD8
:10035B009508402DAE0AAF0BBEFB06BFFE0343B1A3
:10036B003043B701758F01850B82850A83E511F048
:10037B00E4F58F53B7FE75B111050BE50B70020554
:10038B000A050C80A61209CF1209CD8F0EAD0EAF48
:10039B000D1209B68F11E5112512700AE50F6401D4
:0603AB00600302029C2227
:0103B1002229
:0604EB008B4A8A4B894C8C
:1004F1007554FF75550A755666755101755200752B
:100501005350E4F550F54FF54EF54DE47F2BFEFDCC
:10051100FCAB50AA4FA94EA84DC312066C5030AF88
:1005210050E4FBFD120A6F7851E475F0011206C820
:10053100EF12064DAF50AE4FAD4EAC4DE47B01FA1C
:10054100F9F812065F8F508E4F8D4E8C4D80BCABEB
:1005510054AA55A956120607FF900050E06F706229
:10056100900001120620FF900051E06F705490003E
:1005710002120620FF900052E06F704690000312B5
:100581000620FF900053E06F70389000041206209F
:10059100FF900054E06F702A900005120620FF9032
:1005A1000055E0B5071C900006120620FF9000568A
:1005B100E0B5070E900007120620FF900057E06F8C
:1005C10060037F0022AB4AAA4BA94C120607FF9099
:1005D100005FE06F702A900001120620FF9000601A
:1005E100E0B5071C900002120620FF900061E0B503
:1005F100070E900003120620FF900062E06F600377
:050601007F00227F01D3
:0106060022D1
:1008F200E48F34F533F532F531AE33AD32AC3178C5
:10090200081206958F348E338D328C31783512066B
:01091200A83C
:080913008F628E618D608C5F24
:10091B00AA077808120682A907AF62AE61AD60AC78
:0F092B005F7810120682AB07AF02AD01120A6FA0
:01093A00229A
:0400A6008E218F22F6
:1000AA00E4F526F527F534F533F532F531F538F56B
:1000BA0037F536F535F53CF53BF53AF53975382B14
:1000CA00F537F536F535F527F526F52CE4F52BE564
:1000DA0026643A600712090E8F2680F3E53C240154
:1000EA00FFE4353BFEE4353AFDE435398F3C8E3B7F
:1000FA008D3AF53912090E8F2612090E1209B08FA0
:10010A002985292B12090E8F2612090E1209B0E42D
:10011A008F30F52FF52EF52DEF252BF52BAE2FADC4
:10012A002EAC2D78081206958F308E2F8D2E8C2DA1
:10013A0012090E8F2612090E1209B0E5304FFFE59B
:10014A002FFEE52EFDE52D8F308E2F8D2EF52D8E6F
:10015A00238F24EF252BF52B12090E8F2612090E59
:10016A001209B08F28E528252BF52BE528640470A1
:10017A003812090E8F2612090E1209B01208F28FD0
:10018A002612090E1209B0E5344FFFE533FEE532B7
:10019A00FDE5318F348E338D32F531FC781012063D
:1001AA00958F348E338D328C31E528640270381283
:1001BA00090E8F2612090E1209B01208F28F2612A2
:1001CA00090E1209B0E5344FFFE533FEE532FDE5CD
:1001DA00318F348E338D32F531FC78041206958FC7
:1001EA00348E338D328C31E5342524F524E53335CC
:1001FA0023F523E5287058F525E525C39529504FA1
:10020A0012090E8F2612090E1209B08F2AE52A2525
:10021A002BF52BC3E5249522E5239521402DAE230A
:10022A00AF24BEFB06BFFE0343B13043B701758F4F
:10023A0001852482852383E52AF0E4F58F53B7FEEE
:10024A0075B1110524E52470020523052580AA123B
:10025A00090E8F2612090E1209B08F2AE52A252BBC
:0C026A00700AE528640160030200D6223F
:010276002265
:0500060032323341001D
:02001E00C1031C
:100A1C0090007BE584F075840F75E107D2FA75E3DD
:070A2C00C075A4FFE0F58492
:010A330022A0
:100A4900E4F584F5BA75BB0475BCC075E880F58416
:040A590075D103222E
:030016000209EAF2
:10093B00AF84120A1C120A49E4F584FDFC0DBD00BC
:10094B00010CBC27F8BD11F5C2EDD2EC30EDFDAEBC
:0B095B00BFEEFD8F84ED6002C322D3CD
:01096600226E
:10082D00C200C201C20275FFDE75FFAD12093B9217
:10083D000030005E1200167BFF7A0079061203B2BB
:10084D00EF24FF92013001147D007CCC7F007E40AF
:10085D001209677F007E4012027780237BFF7A00AA
:10086D0079061204EBEF24FF92023002127D007C18
:10087D00CC7F007E401209677F007E401200A6E407
:10088D00FFFE0FBF00010EBE27F8BF10F5E4F58483
:05089D00F5C002000E91
:04000E00024000228A
:01FBFE00FE08
:0300000002079361
:03000300025003A5
:03000B000250069A
:030013000250098F
:03001B0002500C84
:0300230002500F79
:03002B000250126E
:0300330002501563
:03003B0002501858
:0300430002501B4D
:03004B0002501E42
:0300530002502137
:03005B000250242C
:0300630002502721
:03006B0002502A16
:0300730002502D0B
:03007B0002503000
:03008300025033F5
:03008B00025036EA
:03009300025039DF
:03009B0002503CD4
:0300A30002503FC9
:10079300787FE4F6D8FD9000007F007E20E4F0A38C
:0A07A300DFFCDEFA7581620207E850
:1008A200E590540C23C0E0740AC0E0C082C0830209
:1008B2000A00E590540C23C0E0740AC0E0C082C074
:1008C20083020A08E590540C23C0E0740AC0E0C019
:1008D20082C083020A10E590540C23C0E0740AC05F
:0808E200E0C082C083020A1885
:040A00005390F322FA
:070A080043900C5390F7220C
:070A100043900C5390FB2200
:040A180043900C22D9
:0708EA00EFC403900A007344
:1007AD0002082DE493A3F8E493A34003F68001F22D
:1007BD0008DFF48029E493A3F85407240CC8C3334D
:1007CD00C4540F4420C8834004F456800146F6DF1C
:1007DD00E4800B010204081020408090001EE47E8E
:1007ED00019360BCA3FF543F30E509541FFEE49311
:1007FD00A360010ECF54C025E060A840B8E493A3D8
:10080D00FAE493A3F8E493A3C8C582C8CAC583CA02
:10081D00F0A3C8C582C8CAC583CADFE9DEE780BEBA
:0100200000DF
:10060700BB010689828A83E0225002E722BBFE02F1
:09061700E32289828A83E4932224
:10062000BB010CE58229F582E5833AF583E022508F
:1006300006E92582F8E622BBFE06E92582F8E222D9
:0D064000E58229F582E5833AF583E49322F3
:10064D00BB010689828A83F0225002F722BBFE018C
:02065D00F32286
:0D065F00EF2BFFEE3AFEED39FDEC38FC22EA
:10066C00EB9FF5F0EA9E42F0E99D42F0EC6480C805
:06067C0064809845F022A5
:10068200E8600FECC313FCED13FDEE13FEEF13FF56
:03069200D8F1227A
:10069500E8600FEFC333FFEE33FEED33FDEC33FCC3
:0306A500D8F12267
:1006A8007401FF3395E0FEFDFC080808E6CF2FF63D
:1006B80018E6CE3EF618E6CD3DF618E6CC3CF62216
:1006C800FAE6FB0808E6F925F0F618E6CA3AF62233
:10098E00EF7E0024D0B40A00401624F9B40A0040C9
:10099E000CB41000400A24E0B41000400374FFFEB3
:0209AE00FF2226
:00000001FF
